:020000040000FA
:10000000BD28A4003608840034082220841300058B
:100010002C1C340603191F282408031D17282A083E
:10002000FF3E031C20280A3048202A082028240AE2
:10003000FF3003191F28240B1F282B082028AD0987
:10004000AD0CB82884178004B82800308A0028082E
:1000500007392D3E03188A0A820001340234043421
:1000600008341034203440348034A000A00DA00D9A
:10007000200D3839C1389F000030A10032305620A1
:100080001F151F1941281E08A10083161E08B82835
:10009000A301A200FF30A207031CA307031CB8287A
:1000A0000330A100DF3056204A28A101E83EA0001D
:1000B000A109FC30031C5F28A00703185C28A007D7
:1000C0006400A10F5C2820186528A01C6928000086
:1000D00069280800A8002520A001A101A81DA000F2
:1000E000A819A1002008B828013EA7000A30A200E4
:1000F000A3018620A70B7928240808000310A10C6F
:10010000A00CFF3E03187E282008B828A501A401F2
:100110001030A600210DA40DA50D2208A40223086D
:10012000031C230FA50203189C282208A4072308F8
:100130000318230FA5070310A00DA10DA60B8A28F5
:100140002008B8281030A800A101A001A70CA60C17
:10015000031CB0282208A00723080318230FA107B7
:10016000A10CA00CA50CA40CA80BA6282408B82848
:10017000831303138312640008008316FF30850085
:1001800082309F0086010F308700963083128A01EB
:1001900048208A110A12ED214908A100023C8A1167
:1001A0000A12031CEC28A10D8A110A12DF20A000FC
:1001B00021108A110A12DF208A00200882000030F4
:1001C0008A002108E63E03188A0A82000034EE34D1
:1001D00001347F340134B6348A01C92800308A01E1
:1001E0003520BA002108BB0001303A07C2003B08A5
:1001F0000318013EC3004208A6004308A700F430DC
:10020000A2000130A3008A01A2202508C200200814
:10021000C3004208A0004308A10002308A018120E7
:10022000BA002108BB003A08A6003B08A70004302A
:10023000A200A3018A01A220BC002508BD00C13094
:10024000CF008A110A1224298A110A1229218A014F
:10025000C928CC01640004304C028A110A12031828
:100260005C293C08A0003D08A1004C088A017420CC
:10027000CD008A110A125D2101308A014820043024
:100280004C07D00064005008073C8A110A12031D75
:100290004B294F08860064005008053C8A110A1259
:1002A000031D5329861350088A016A208700CC0A4F
:1002B0008A110A12031D2A29080087014D080B3CE8
:1002C0008A110A12031C7E298A110A126B218600E8
:1002D0008A110A127E2901308A004D08723E0318E5
:1002E0008A0A8200C034F934A434B0349934923488
:1002F0008234F83480349034BF34FF340800DC306A
:10030000CF003E08BC003F08BD00C5010730B60065
:100310000130B400AC01FF30AA000530AB00AD01E4
:1003200045088A010120C5008A110A1203189B2979
:10033000BE0A0319BF0AC6010730B6000230B40076
:10034000AC01FF30AA000530AB00AD0146088A01C0
:100350000120C6008A110A120318B4290130BE0216
:100360000030031C013EBF028A012429E330CF0084
:100370004008BC004108BD00C7010730B60001308D
:10038000B400AC01FF30AA000530AB00AD01470856
:100390008A010120C7008A110A120318D229C00A53
:1003A0000319C10AC8010730B6000230B400AC011D
:1003B000FF30AA000530AB00AD0148088A010120DA
:1003C000C8008A110A120318EB290130C00200305C
:1003D000031C013EC1028A012429C4010730B60072
:1003E0000830B400AC01FF30AA000A30AB00AD0108
:1003F00044088A010120C4008A110A120318102A35
:1004000064008A110A124E180F2AC90A64004908AA
:10041000043C8A110A12031D0E2AC9014E14080059
:0A0420004E10080063008A01122A42
:02400E007D3FF4
:00000001FF
